:020000040800F2
:1000000000C0002071400008254000082940000879
:100010002D40000831400008354000080000000075
:10002000000000000000000000000000394000084F
:100030003D40000800000000414000084540000825
:10004000C1400008C1400008C1400008C14000088C
:10005000C1400008C1400008C1400008C14000087C
:10006000C1400008C1400008C1400008C138000874
:10007000C1400008C1400008C1400008C14000085C
:100080005140000861400008C1400008C14000081C
:10009000C1400008C1400008C1400008C14000083C
:1000A000C1400008C1400008C1400008C14000082C
:1000B000C1400008C1400008C1400008C14000081C
:1000C000C1400008C1400008C1400008C14000080C
:1000D000C1400008C1400008C1400008C1400008FC
:1000E000C1400008C1400008C1400008C1400008EC
:1000F000C1400008C1400008C1400008C1400008DC
:10010000C1400008C1400008C1400008C1400008CB
:10011000C1400008C1400008C1400008C1400008BB
:10012000C1400008C1400008C1400008C1400008AB
:1001300000000000000000000000000000000000BF
:1001400000000000000000000000000000000000AF
:10015000000000000000000000000000000000009F
:10016000000000000000000000000000000000008F
:10017000000000000000000000000000000000007F
:10018000000000000000000000000000000000006F
:10019000000000000000000000000000000000005F
:1001A000000000000000000000000000000000004F
:1001B000000000000000000000000000000000003F
:1001C000000000000000000000000000000000002F
:1001D000000000000000000000000000000000001F
:0401E0005FF8E0F1F3
:1001E80010B5054C237833B9044B13B10448AFF369
:1001F80000800123237010BD88000020000000004B
:100208005C49000808B5064B1BB106480649AFF320
:1002180000800648036813B1054B03B1984708BD31
:10022800000000005C4900088C00002088000020C5
:100238000000000081F0004102E000BF83F00043AD
:1002480030B54FEA41044FEA430594EA050F08BF69
:1002580090EA020F1FBF54EA000C55EA020C7FEA2D
:10026800645C7FEA655C00F0E2804FEA5454D4EBAA
:100278005555B8BF6D420CDD2C4480EA020281EA74
:10028800030382EA000083EA010180EA020281EAAC
:100298000303362D88BF30BD11F0004F4FEA0131FE
:1002A8004FF4801C4CEA113102D0404261EB41010D
:1002B80013F0004F4FEA03334CEA133302D0524293
:1002C80063EB430394EA050F00F0A780A4F101044F
:1002D800D5F1200E0DDB02FA0EFC22FA05F2801889
:1002E80041F1000103FA0EF2801843FA05F359416F
:1002F8000EE0A5F120050EF1200E012A03FA0EFCEE
:1003080028BF4CF0020C43FA05F3C01851EBE37117
:1003180001F0004507D54FF0000EDCF1000C7EEB34
:1003280000006EEB0101B1F5801F1BD3B1F5001F72
:100338000CD349085FEA30004FEA3C0C04F1010491
:100348004FEA445212F5800F80F09A80BCF1004FBA
:1003580008BF5FEA500C50F1000041EB045141EA3C
:10036800050130BD5FEA4C0C404141EB010111F43D
:10037800801FA4F10104E9D191F0000F04BF0146E8
:100388000020B1FA81F308BF2033A3F10B03B3F1C6
:1003980020020CDA0C3208DD02F1140CC2F10C0256
:1003A80001FA0CF021FA02F10CE002F11402D8BFB4
:1003B800C2F1200C01FA02F120FA0CFCDCBF41EA80
:1003C8000C019040E41AA2BF01EB0451294330BD4F
:1003D8006FEA04041F3C1CDA0C340EDC04F114042C
:1003E800C4F1200220FA04F001FA02F340EA030003
:1003F80021FA04F345EA030130BDC4F10C04C4F149
:10040800200220FA02F001FA04F340EA0300294628
:1004180030BD21FA04F0294630BD94F0000F83F472
:10042800801306BF81F480110134013D4EE77FEA55
:10043800645C18BF7FEA655C29D094EA050F08BFA1
:1004480090EA020F05D054EA000C04BF1946104682
:1004580030BD91EA030F1EBF0021002030BD5FEAC6
:10046800545C05D14000494128BF41F0004130BDEE
:1004780014F580043CBF01F5801130BD01F0004542
:1004880045F0FE4141F470014FF0000030BD7FEAB5
:10049800645C1ABF194610467FEA655C1CBF0B46B0
:1004A800024650EA013406BF52EA033591EA030FC7
:1004B80041F4002130BD00BF90F0000F04BF0021BF
:1004C800704730B54FF4806404F132044FF00005F2
:1004D8004FF0000150E700BF90F0000F04BF00216B
:1004E800704730B54FF4806404F1320410F00045D1
:1004F80048BF40424FF000013EE700BF42004FEACC
:10050800E2014FEA31014FEA02701FBF12F07F4348
:1005180093F07F4F81F06051704792F0000F14BF45
:1005280093F07F4F704730B54FF4607401F0004589
:1005380021F0004120E700BF50EA010208BF7047E0
:1005480030B54FF000050AE050EA010208BF7047D5
:1005580030B511F0004502D5404261EB41014FF43E
:10056800806404F132045FEA915C3FF4DCAE4FF042
:1005780003025FEADC0C18BF03325FEADC0C18BF29
:10058800033202EBDC02C2F1200300FA03FC20FA7A
:1005980002F001FA03FE40EA0E0021FA02F11444C7
:1005A800C1E600BF70B54FF0FF0C4CF4E06C1CEADC
:1005B80011541DBF1CEA135594EA0C0F95EA0C0F51
:1005C80000F0DEF82C4481EA030621EA4C5123EAC4
:1005D8004C5350EA013518BF52EA033541F48011F3
:1005E80043F4801338D0A0FB02CE4FF00005E1FBA6
:1005F80002E506F00042E0FB03E54FF00006E1FBF0
:1006080003569CF0000F18BF4EF0010EA4F1FF0432
:10061800B6F5007F64F5407404D25FEA4E0E6D4172
:1006280046EB060642EAC62141EA55514FEAC52083
:1006380040EA5E504FEACE2EB4F1FD0C88BFBCF5FF
:10064800E06F1ED8BEF1004F08BF5FEA500E50F1B0
:10065800000041EB045170BD06F0004646EA010176
:1006680040EA020081EA0301B4EB5C04C2BFD4EBA8
:100678000C0541EA045170BD41F480114FF0000EA1
:10068800013C00F3AB8014F1360FDEBF002001F00F
:10069800004170BDC4F10004203C35DA0C341BDC89
:1006A80004F11404C4F1200500FA05F320FA04F05B
:1006B80001FA05F240EA020001F0004221F000418F
:1006C80010EBD37021FA04F642EB06015EEA430E02
:1006D80008BF20EAD37070BDC4F10C04C4F1200532
:1006E80000FA04F320FA05F001FA04F240EA0200E5
:1006F80001F0004110EBD37041F100015EEA430EB6
:1007080008BF20EAD37070BDC4F1200500FA05F2D5
:100718004EEA020E20FA04F301FA05F243EA020354
:1007280021FA04F001F0004121FA04F220EA020063
:1007380000EBD3705EEA430E08BF20EAD37070BDA9
:1007480094F0000F0FD101F00046400041EB010189
:1007580011F4801F08BF013CF7D041EA060195F06B
:10076800000F18BF704703F00046520043EB030325
:1007780013F4801F08BF013DF7D043EA0603704712
:1007880094EA0C0F0CEA135518BF95EA0C0F0CD01D
:1007980050EA410618BF52EA4306D1D181EA030163
:1007A80001F000414FF0000070BD50EA410606BF5D
:1007B8001046194652EA430619D094EA0C0F02D1A2
:1007C80050EA013613D195EA0C0F05D152EA0336E7
:1007D8001CBF104619460AD181EA030101F0004105
:1007E80041F0FE4141F470014FF0000070BD41F04E
:1007F800FE4141F4780170BD70B54FF0FF0C4CF428
:10080800E06C1CEA11541DBF1CEA135594EA0C0F46
:1008180095EA0C0F00F0A7F8A4EB050481EA030E93
:1008280052EA03354FEA013100F088804FEA03337A
:100838004FF0805545EA131343EA12634FEA022248
:1008480045EA111545EA10654FEA00260EF0004109
:100858009D4208BF964244F1FD0404F5407402D25B
:100868005B084FEA3202B61A65EB03055B084FEAEC
:1008780032024FF480104FF4002CB6EB020E75EBE9
:10088800030E22BFB61A754640EA0C005B084FEA11
:100898003202B6EB020E75EB030E22BFB61A75468E
:1008A80040EA5C005B084FEA3202B6EB020E75EBD9
:1008B800030E22BFB61A754640EA9C005B084FEA51
:1008C8003202B6EB020E75EB030E22BFB61A75465E
:1008D80040EADC0055EA060E18D04FEA051545EA4D
:1008E80016754FEA06164FEAC30343EA52734FEAF6
:1008F800C2025FEA1C1CC0D111F4801F0BD141EA6F
:1009080000014FF000004FF0004CB6E711F4801FD3
:1009180004BF01430020B4F1FD0C88BFBCF5E06FB3
:100928003FF6AFAEB5EB030C04BFB6EB020C5FEAC3
:10093800500C50F1000041EB045170BD0EF0004E18
:100948004EEA113114EB5C04C2BFD4EB0C0541EA4A
:10095800045170BD41F480114FF0000E013C90E647
:1009680045EA060E8DE60CEA135594EA0C0F08BF0B
:1009780095EA0C0F3FF43BAF94EA0C0F0AD150EA0A
:1009880001347FF434AF95EA0C0F7FF425AF10469D
:1009980019462CE795EA0C0F06D152EA03353FF4C5
:1009A800FDAE1046194622E750EA410618BF52EA42
:1009B80043067FF4C5AE50EA41047FF40DAF52EA16
:1009C80043057FF4EBAE12E74FF0FF3C06E000BFB3
:1009D8004FF0010C02E000BF4FF0010C4DF804CDC0
:1009E8004FEA410C7FEA6C5C4FEA430C18BF7FEA80
:1009F8006C5C1BD001B050EA410C0CBF52EA430CAE
:100A080091EA030F02BF90EA020F0020704710F12D
:100A1800000F91EA030F58BF994208BF90422CBFBC
:100A2800D8176FEAE37040F0010070474FEA410CB5
:100A38007FEA6C5C02D150EA013C07D14FEA430CD3
:100A48007FEA6C5CD6D152EA033CD3D05DF8040B44
:100A5800704700BF8446104662468C461946634676
:100A680000E000BF01B5FFF7B7FF002848BF10F14D
:100A7800000F01BD4DF808EDFFF7F4FF0CBF012092
:100A880000205DF808FB00BF4DF808EDFFF7EAFF0E
:100A980034BF012000205DF808FB00BF4DF808EDC9
:100AA800FFF7E0FF94BF012000205DF808FB00BFBE
:100AB8004DF808EDFFF7CEFF94BF012000205DF848
:100AC80008FB00BF4DF808EDFFF7C4FF34BF012055
:100AD80000205DF808FB00BF4FEA410212F5001242
:100AE80015D211D56FF47873B3EB625212D94FEA6D
:100AF800C12343F0004343EA505311F0004F23FA57
:100B080002F018BF404270474FF00000704750EAAB
:100B1800013005D111F0004008BF6FF00040704768
:100B28004FF00000704700BF4FEA4102B2F1E043C6
:100B380024BFB3F5001CDCF1FE5C0DD901F0004CBC
:100B48004FEAC0024CEA5070B2F1004F40EB83000C
:100B580008BF20F00100704711F0804F21D113F138
:100B68003872BCBF01F00040704741F480114FEA71
:100B78005252C2F11802C2F1200C10FA0CF320FAFA
:100B880002F018BF40F001004FEAC1234FEAD32317
:100B980003FA0CFC40EA0C0023FA02F34FEA430381
:100BA800CCE77FEA625307D150EA01331EBF4FF00A
:100BB800FE4040F44000704701F0004040F0FE4025
:100BC80040F40000704700BF80F0004002E000BF22
:100BD80081F0004142001FBF5FEA410392EA030F20
:100BE8007FEA226C7FEA236C6AD04FEA1262D2EB6A
:100BF8001363C1BFD218414048404140B8BF5B426F
:100C0800192B88BF704710F0004F40F4000020F007
:100C18007F4018BF404211F0004F41F4000121F01D
:100C28007F4118BF494292EA030F3FD0A2F1010267
:100C380041FA03FC10EB0C00C3F1200301FA03F1A5
:100C480000F0004302D5494260EB4000B0F5000FC8
:100C580013D3B0F1807F06D340084FEA310102F187
:100C68000102FE2A51D2B1F1004F40EBC25008BF39
:100C780020F0010040EA03007047490040EB000003
:100C880010F4000FA2F10102EDD1B0FA80FCACF132
:100C9800080CB2EB0C0200FA0CF0AABF00EBC25031
:100CA80052421843BCBFD0401843704792F0000F1F
:100CB80081F4000106BF80F400000132013BB5E772
:100CC8004FEA41037FEA226C18BF7FEA236C21D0E8
:100CD80092EA030F04D092F0000F08BF084670474D
:100CE80090EA010F1CBF0020704712F07F4F04D11B
:100CF800400028BF40F00040704712F100723CBF2E
:100D080000F50000704700F0004343F0FE4040F457
:100D1800000070477FEA226216BF08467FEA236315
:100D28000146420206BF5FEA412390EA010F40F400
:100D3800800070474FF0000304E000BF10F000434C
:100D480048BF40425FEA000C08BF704743F0964333
:100D580001464FF000001CE050EA010208BF70474E
:100D68004FF000030AE000BF50EA010208BF7047D5
:100D780011F0004302D5404261EB41015FEA010CEA
:100D880002BF84460146002043F0B64308BFA3F1E2
:100D98008053A3F50003BCFA8CF2083AA3EBC253C4
:100DA80010DB01FA02FC634400FA02FCC2F12002E3
:100DB800BCF1004F20FA02F243EB020008BF20F01A
:100DC8000100704702F1200201FA02FCC2F1200280
:100DD80050EA4C0021FA02F243EB020008BF20EA75
:100DE800DC7070474FF0FF3C06E000BF4FF0010C8D
:100DF80002E000BF4FF0010C4DF804CD4FEA40026D
:100E08004FEA41037FEA226C18BF7FEA236C11D0B6
:100E180001B052EA530C18BF90EA010F58BFB2EB69
:100E2800030088BFC81738BF6FEAE17018BF40F0E9
:100E3800010070477FEA226C02D15FEA402C05D19D
:100E48007FEA236CE4D15FEA412CE1D05DF8040B22
:100E5800704700BF844608466146FFE70FB5FFF7B5
:100E6800C9FF002848BF10F1000F0FBD4DF808ED6D
:100E7800FFF7F4FF0CBF012000205DF808FB00BF5E
:100E88004DF808EDFFF7EAFF34BF012000205DF8B8
:100E980008FB00BF4DF808EDFFF7E0FF94BF012005
:100EA80000205DF808FB00BF4DF808EDFFF7D2FF02
:100EB80094BF012000205DF808FB00BF4DF808ED45
:100EC800FFF7C8FF34BF012000205DF808FB00BF12
:100ED80082B0084B1A68084BA3FB02135B0A00FB9D
:100EE80003F0019000BF019B5A1E0192002BF9D11B
:100EF80002B0704700000020D34D62102DE9F04188
:100F080082B00446036813F0010F6ED0A24B5B68F1
:100F180003F00C03042B0AD09F4B5B6803F00C030F
:100F2800082B0DD19C4B5B6813F4803F08D09A4B7B
:100F38001B6813F4003F58D06368002B55D1C1E1FA
:100F48006368B3F5803F08D103F1804303F5883324
:100F58001A6842F480321A6026E063B903F18043CC
:100F680003F504331A6822F480321A601A6822F4EE
:100F780080221A6018E0B3F5A02F0CD103F180434A
:100F8800A3F53C331A6842F480221A601A6842F4C6
:100F980080321A6008E0804B1A6822F480321A60A6
:100FA8001A6822F480221A6063687BB101F03AF86B
:100FB8000646794D05E001F035F8801B642800F2FB
:100FC80083812B6813F4003FF5D00EE001F02AF876
:100FD8000646714D05E001F025F8801B642800F2F3
:100FE80075812B6813F4003FF5D1236813F0020FC5
:100FF80050D0694B5B6813F00C0F0AD0664B5B68E6
:1010080003F00C03082B16D1634B5B6813F4803F85
:1010180011D1614B1B6813F0020F03D02369012B18
:1010280040F056815C4B196821F0F801626941EA89
:10103800C2021A602EE02369D3B10122574B1A600D
:1010480000F0F0FF0646544D05E000F0EBFF801B72
:10105800022800F23F812B6813F0020FF5D04E4BA7
:10106800196821F0F801626941EAC2021A6011E0C8
:1010780000224A4B1A6000F0D5FF0646464D05E0AF
:1010880000F0D0FF801B022800F226812B6813F0A5
:10109800020FF5D1236813F0080F29D0A369ABB16B
:1010A80001223F4B1A6000F0BDFF06463A4D05E0AD
:1010B80000F0B8FF801B022800F210816B6A13F061
:1010C800020FF5D00120FFF703FF11E00022344B97
:1010D8001A6000F0A7FF06462F4D05E000F0A2FFBA
:1010E800801B022800F2FC806B6A13F0020FF5D116
:1010F800236813F0040F00F08C80274BDB6913F092
:10110800805F0BD1244BDA6942F08052DA61DB69E7
:1011180003F080530193019B012500E00025214B3A
:101128001B6813F4807F13D11E4B1A6842F4807237
:101138001A6000F077FF07461A4E05E000F072FFCC
:10114800C01B642800F2CE80336813F4807FF5D08A
:10115800E368012B05D1104B1A6A42F001021A62AA
:101168002BE063B903F1804303F504331A6A22F0D4
:1011780001021A621A6A22F004021A621DE0052BA3
:1011880012D1054B1A6A42F004021A621A6A42F036
:1011980001021A6211E000BF001002400000424242
:1011A8008004424200700040574B1A6A22F0010244
:1011B8001A621A6A22F004021A62E36893B100F014
:1011C80031FF8046504E41F2883706E000F02AFF92
:1011D800C8EB0000B84200F28780336A13F0020FB0
:1011E800F4D010E000F01EFF8046474E41F28837E9
:1011F80005E000F017FFC8EB0000B84276D8336A64
:1012080013F0020FF5D125B13F4BDA6922F0805275
:10121800DA61E369002B6BD03B4A526802F00C029A
:10122800082A67D0022B3AD10022384B1A6000F006
:10123800F9FE0646344D04E000F0F4FE801B022857
:101248005AD82B6813F0007FF6D1236AB3F5803F94
:1012580009D103F1804303F58833596821F400313B
:10126800A2680A435A60284B596821F47411206A0D
:10127800626A02430A435A600122244B1A6000F052
:10128800D1FE0546204C04E000F0CCFE401B0228AD
:1012980034D8236813F0007FF6D0002031E0002214
:1012A8001A4B1A6000F0BEFE0546174C04E000F029
:1012B800B9FE401B022823D8236813F0007FF6D11B
:1012C80000201EE001201CE003201AE0032018E0A3
:1012D800012016E0032014E0032012E0032010E0B0
:1012E80003200EE003200CE003200AE0032008E0BE
:1012F800002006E0012004E0032002E0032000E0D3
:10130800032002B0BDE8F0810010024060004242B4
:1013180030B486B0164D02AC28686968AA68EB68D4
:101328000FC42B8AADF80430124B5B6803F00C0233
:10133800082A19D1C3F3834206A90A4412F8102CCB
:1013480013F4803F0CD00B4B5B68C3F340430B4452
:1013580013F8143C0848B0FBF3F002FB00F004E07B
:10136800064800FB02F000E0034806B030BC7047B6
:10137800744900080010024000127A0000093D007C
:101388002DE9F04104460D46614B1B6803F0070345
:101398008B420BD25E4B1A6822F007020A431A608E
:1013A8001B6803F007038B4240F09980236813F011
:1013B800020F06D0574B596821F0F001A2680A4382
:1013C8005A60236813F0010F50D06368012B05D1D0
:1013D800504A126812F4003F0DD183E0022B05D168
:1013E8004C4A126812F0007F05D17EE0494A126823
:1013F80012F0020F7CD0474A516821F003010B43D9
:10140800536000F00FFE06466368012B0FD105E01C
:1014180000F008FE801B404503D96CE03D4F41F2C7
:1014280088387B6803F00C03042BF1D11EE0022BF3
:1014380015D105E000F0F6FD801B404503D95DE0BD
:10144800344F41F288387B6803F00C03082BF1D144
:101458000CE000F0E7FD801B404503D951E02D4F1B
:1014680041F288387B6813F00C0FF2D1284B1B68C7
:1014780003F00703AB420AD9254B1A6822F007028A
:101488002A431A601B6803F00703AB423CD1236868
:1014980013F0040F06D01F4B596821F4E061E2688D
:1014A8000A435A60236813F0080F07D0194B5A688B
:1014B80022F46052216942EAC1025A60FFF728FF0C
:1014C800144B5B68C3F30313134AD35CD840134A25
:1014D8001060002000F076FD0020BDE8F0810120BA
:1014E800BDE8F0810120BDE8F0810120BDE8F08170
:1014F8000120BDE8F0810320BDE8F0810320BDE8AC
:10150800F0810320BDE8F0810120BDE8F08100BF33
:101518000020024000100240884900080000002016
:10152800014B1868704700BF0000002008B5FFF79E
:10153800F7FF044B5B68C3F30223034AD35CD8402C
:1015480008BD00BF001002409849000808B5FFF721
:10155800E7FF044B5B68C3F3C223034AD35CD8405C
:1015680008BD00BF001002409849000830B4036A63
:1015780023F001030362026A4368856925F0730555
:101588000C68254322F002028C682243104CA042CA
:1015980003D004F50064A04205D122F00802CC680B
:1015A800224322F004020A4CA04203D004F500644E
:1015B800A04205D123F440734C6923438C6923432B
:1015C800436085614B684363026230BC704700BF6B
:1015D800002C014030B4036A23F480730362026A6A
:1015E8004368C56925F073050C68254322F4007229
:1015F8008C6842EA0422124CA04203D004F500642D
:10160800A04206D122F40062CC6842EA042222F405
:1016180080620B4CA04203D004F50064A04207D1BD
:1016280023F440534C6943EA04138C6943EA0413D6
:101638004360C5614B68C363026230BC704700BF3A
:10164800002C014030B4036A23F480530362056A16
:101658004368C26922F4E6420C6842EA042425F48D
:1016680000558A6845EA0232094DA84203D005F5BB
:101678000065A84204D123F480434D6943EA8513E9
:101688004360C4614B680364026230BC704700BFAA
:10169800002C014010B4036A046A24F001040462B7
:1016A800846924F0F00444EA021223F00A0319437F
:1016B800826101625DF8044B704700BF10B4036A91
:1016C80023F0100303628469036A24F4704444EA33
:1016D800023223F0A00343EA0111826101625DF83E
:1016E800044B704710B4846824F47F4442EA03230F
:1016F80019430C4384605DF8044B704710B50B46E2
:101708000268946824F070044968214321F00704B2
:101718001968214391605A68502A1FD002D8402A7C
:101728000BD010BD602A1FD0702A22D10068D9685A
:101738009A681B69FFF7D6FF10BD0268116A146A20
:1017480024F0010414620268946924F0F0041B690F
:1017580044EA031393610368196210BD006899682D
:101768001A69FFF797FF10BD006899681A69FFF7B3
:10177800A5FF10BD704700BF38B5044690F83C304F
:10178800012B17D0012580F83C50022380F83D300A
:10179800FFF7B4FF2368DA6822F04002DA602368B2
:1017A800DA6822F48042DA6084F83D50002084F838
:1017B8003C0038BD022038BD0368244A904212D04C
:1017C80002F5006290420ED0B0F1804F0BD0A2F526
:1017D8009832904207D002F58062904203D002F519
:1017E8008062904203D123F070034A681343174A7A
:1017F800904212D002F5006290420ED0B0F1804FB4
:101808000BD0A2F59832904207D002F58062904240
:1018180003D002F58062904203D123F44073CA6872
:10182800134323F080034A691A4302608B68C3623A
:101838000B688362054B984203D003F50063984216
:1018480001D10B690363012343617047002C0140F8
:1018580010B50446B0B190F83D3013F0FF0F04D135
:10186800002380F83C30FFF785FF022384F83D30E1
:10187800214651F8040BFFF79FFF012384F83D3000
:10188800002010BD012010BD30B4036A23F01003FE
:101898000362026A4368856925F4E6450C6845EAEF
:1018A800042522F020028C6842EA0412114CA0425E
:1018B80003D004F50064A04206D122F08002CC686F
:1018C80042EA041222F040020A4CA04203D004F576
:1018D8000064A04207D123F440634C6943EA8403BF
:1018E8008C6943EA8403436085614B6883630262C1
:1018F80030BC7047002C014038B504460D4690F8BE
:101908003C30012B64D0012380F83C30022380F85E
:101918003D300C2A55D8DFE802F0075454541A54C5
:1019280054542E54545441000068FFF71FFE236896
:101938009A6942F008029A6123689A6922F00402BF
:101948009A61236899692A690A439A6139E00068AB
:10195800FFF79AFF23689A6942F400629A61236844
:101968009A6922F480629A6123689A69296942EA2D
:1019780001229A6125E00068FFF72CFE2368DA69E6
:1019880042F00802DA612368DA6922F00402DA61B7
:101998002368D9692A690A43DA6112E00068FFF707
:1019A80051FE2368DA6942F40062DA612368DA6971
:1019B80022F48062DA612368DA69296942EA01223D
:1019C800DA61012384F83D30002084F83C0038BDFA
:1019D800022038BD10B401238B40046A24EA0303B3
:1019E8000362036A8A40134303625DF8044B70473D
:1019F80010B5044600680122FFF7ECFF23680C4A83
:101A0800934205D002F50062934203D1012202E01D
:101A1800012200E000221AB15A6C42F400425A64D2
:101A280023681A6842F001021A60002010BD00BF46
:101A3800002C014010B404238B40046A24EA0303F9
:101A48000362036A8A40134303625DF8044B7047DC
:101A580010B5044600680422FFF7ECFF23685A6CAF
:101A680042F400425A6423681A6842F001021A607C
:101A7800002010BD90F83C30012B22D0012380F8C3
:101A88003C30CB6823F440728B68134323F48062A4
:101A98004B681A4322F400620B681A4322F48052FE
:101AA8000B691A4322F400524B691A43896922F4DC
:101AB80040420A4303685A64002380F83C301846C1
:101AC80070470220704700BF30B490F83C30012BBB
:101AD80020D0012380F83C30022280F83D200268A3
:101AE800546824F070045460026855680C682C43EC
:101AF80054600268946824F08004946002689468D2
:101B080049682143916080F83D30002380F83C30DB
:101B1800184600E0022030BC704700BF10B490F8AF
:101B28002430012B21D0012380F8243003689A68DF
:101B380012F0010F0FD10F4A926812F0010F0AD16B
:101B48000D4A934207D15C6824F470240A68224342
:101B58005A60002304E0836A43F020038362012370
:101B6800002280F82420184600E002205DF8044B8B
:101B7800704700BF002801400024014000F0070022
:101B8800064AD36823F4E0631B041B0C43EA0023D2
:101B980043F0BF6343F40033D360704700ED00E0C7
:101BA80030B4164BDB68C3F30223C3F10705042DD9
:101BB80028BF04251C1D062C01D9033B00E0002387
:101BC800012404FA05F5013D2940994004FA03F37C
:101BD800013B1A400A43002806DA00F00F00120100
:101BE800D2B2074B1A5407E01201D2B200F160409A
:101BF80000F5614080F8002330BC704700ED00E03C
:101C080014ED00E0420900F01F00012303FA00F080
:101C1800014B43F82200704700E100E00138B0F1C1
:101C2800807F0AD2064B5860F021064A82F82310BA
:101C38000020986007221A6070470120704700BF93
:101C480010E000E000ED00E0042805D1054B1A681B
:101C580042F004021A607047024B1A6822F004022C
:101C68001A60704710E000E0704700BF08B5FFF742
:101C7800FBFF08BD2DE9F00F82B000252B46784FF9
:101C8800DFF8E4C1DFF8E481764C8146E1E0012623
:101C98009E400A683240B24240F0DA804868122812
:101CA8002FD00BD8022829D003D868B3012820D018
:101CB80039E0032834D011281DD034E0DFF8B0A172
:101CC800504521D008D8AAF5801A50451CD00AF5ED
:101CD800803A504527D117E0DFF898A1504513D036
:101CE8000AF5803A50450FD0AAF5801A50451AD106
:101CF8000AE0CD6817E0CD68043514E0CD680835F2
:101D080011E0CD680C350EE0886858B1012803D180
:101D1800C9F81060082506E0C9F81460082502E033
:101D2800002500E00425FF2A01D8484601E009F112
:101D38000400FF2A01D89E0002E0A3F10806B600BD
:101D4800D0F800B04FF00F0A0AFA06FA2BEA0A0A8E
:101D580005FA06F64AEA06060660486810F0805F4B
:101D680076D0B86940F00100B861B86900F00100A8
:101D7800019001989808861C5CF826B003F00306C9
:101D8800B6004FF00F0A0AFA06FA2BEA0A0AC1450A
:101D980025D0DFF8E4B0D9451ED00BF5806BD945C6
:101DA80017D00BF5806BD94510D00BF5806BD94552
:101DB80009D00BF5806BD94502D14FF0050B10E027
:101DC8004FF0060B0DE04FF0040B0AE04FF0030B49
:101DD80007E04FF0020B04E04FF0010B01E04FF079
:101DE800000B0BFA06F646EA0A0602304CF82060A9
:101DF800486810F4803F03D020681043206003E057
:101E0800206820EA02002060486810F4003F03D0F0
:101E180060681043606003E0606820EA0200606068
:101E2800486810F4801F03D0A0681043A06003E046
:101E3800A06820EA0200A060486810F4001F03D0E0
:101E4800E0680243E26003E0E06820EA0202E26040
:101E580001330F2B7FF61BAF02B0BDE8F00F7047C0
:101E68000010024000040140000001400008014049
:101E78000000211000003110000C014083680B4263
:101E880001D0012070470020704700BF0AB10161EE
:101E98007047090401617047C3685940C1607047C1
:101EA8002DE9F04182B00446036813F0010F60D0B9
:101EB800404BDB6913F0805F0BD13E4BDA6942F08F
:101EC8008052DA61DB6903F080530193019B01279B
:101ED80000E00027384B1B6813F4807F12D1364B83
:101EE8001A6842F480721A6000F09CF80646324D77
:101EF80004E000F097F8801B642852D82B6813F48C
:101F0800807FF6D02B4B1B6A13F4407325D0626890
:101F180002F440729A4220D0264A136A23F4407091
:101F2800264901250D6000250D60106213F0010F90
:101F380013D000F077F8804605F1804505F50435A3
:101F480041F2883605E000F06DF8C8EB0000B042B9
:101F580029D82B6A13F0020FF5D0164B196A21F411
:101F6800407162680A431A621FB1DA6922F080522E
:101F7800DA61236813F0020F06D00E4B596821F47A
:101F88004041A2680A435A60236813F0100F0CD02E
:101F9800084B5A6822F4800261690A435A6000209B
:101FA80004E0032002E0032000E0002002B0BDE8C6
:101FB800F08100BF0010024000700040400442421F
:101FC800704700BF10B50446074B1868074BA3FBC2
:101FD80000208009FFF722FE4FF0FF302146002243
:101FE800FFF7DEFD002010BD00000020D34D621079
:101FF80008B5074B1A6842F010021A600320FFF771
:10200800BDFD0020FFF7DEFFFFF7DAFF002008BD67
:1020180000200240024B1A6801321A60704700BF64
:10202800E0000020014B1868704700BFE000002066
:1020380030B583B00190FFF7F5FF0546019CB4F178
:10204800FF3F00D00134FFF7EDFF401BA042FAD359
:1020580003B030BD704700BF30B482B00023019395
:1020680090F82430012B00F08980012380F8243077
:102078004B68062B0ED80268546B03EB8303053BB1
:102088001F259D4024EA05050C6804FA03F32B4339
:1020980053631EE00C2B0ED80268146B03EB83030A
:1020A800233B1F259D4024EA05050C6804FA03F329
:1020B8002B4313630DE00268D46A03EB8303413BAF
:1020C8001F259D4024EA05050C6804FA03F32B43F9
:1020D800D3620B68092B0ED90268D46803EB43035B
:1020E8001E3B07259D4024EA05058C6804FA03F386
:1020F8002B43D3600CE00268146903EB4303072504
:102108009D4024EA05058C6804FA03F32B43136108
:102118000B68103B012B27D803681A4A93421DD13C
:102128009A6812F4000F21D19A6842F400029A606A
:102138000B68102B1CD1144B1A68144BA3FB021309
:102148009B0C03EB83035B00019302E0019B013BC3
:102158000193019B002BF9D100220AE0836A43F026
:1021680020038362012204E0002202E0002200E052
:102178000022002380F82430104600E0022002B03C
:1021880030BC7047002401400000002083DE1B4360
:1021980030B583B004460023019303689A6812F0AF
:1021A800010F2ED19A6842F001029A60164B1A6804
:1021B800164BA3FB02139B0C019302E0019B013B0E
:1021C8000193019B002BF9D1FFF72CFF054611E085
:1021D800FFF728FF401B02280CD9A36A43F010031D
:1021E800A362E36A43F00103E362002384F8243026
:1021F800012007E023689B6813F0010FE8D0002056
:1022080000E0002003B030BD0000002083DE1B4347
:1022180010B5044690F82430012B6ED0012380F8C5
:102228002430FFF7B5FF0246002861D1A36A23F4E2
:10223800407323F0010343F48073A3622368304999
:102248008B4205D1A1F58061496811F4702F0ED138
:10225800A16A21F48011A162596811F4806F1CD021
:10226800A16A21F4405141F48051A16215E0A16AAC
:1022780041F48011A16223498B4203D001F58061AA
:102288008B420AD11F49496811F4806F05D0A16AB1
:1022980021F4405141F48051A162A16A11F4805F98
:1022A80004D0E16A21F00601E16201E00021E16267
:1022B800002184F824106FF00201196023689968DE
:1022C80001F46021B1F5602F0DD10D498B4205D184
:1022D800A1F58061496811F4702F04D1996841F41F
:1022E800A001996007E0996841F48011996002E0C3
:1022F800002384F82430104610BD022010BD00BF12
:10230800002801400024014038B5044603689A6853
:1023180012F0010F1DD09A6822F001029A60FFF7AF
:1023280081FE05460EE0FFF77DFE401B022809D915
:10233800A36A43F01003A362E36A43F00103E36274
:10234800012038BD23689B6813F0010FEBD10020F2
:1023580038BD002038BD00BF70B50446002800F025
:102368008680836A23B9C36280F82430FFF772FE3F
:102378002046FFF7C9FFA36A13F0100F71D1002898
:102388006FD1A36A23F4885323F0020343F00203B6
:10239800A36261682368374A934206D1E269B2F5BD
:1023A800402F03D14FF4002200E0E2690A43E568B8
:1023B80042EA4502A168B1F5807F04D0012905D120
:1023C8004FF4807103E04FF4807100E000216669EA
:1023D800012E0FD135B9A569013D41EA453141F4D6
:1023E800006107E0A56A45F02005A562E56A45F0A9
:1023F8000105E5625D6825F469452943596021684E
:102408008D681D4B2B4013438B60A368B3F5807F09
:1024180001D0012B03D12569013D2D0500E00025E0
:102428002368D96A21F470012943D962236899681D
:10243800124B0B409A4208D10023E362A36A23F0AF
:10244800030343F00103A36270BDA36A23F01203E0
:1024580043F01003A362E36A43F00103E36201203F
:1024680070BDA36A43F01003A362012070BD012070
:1024780070BD00BF003C0140FDF7E1FFFE0E1FFFED
:102488000368DA6822F0C002DA60202380F8393065
:10249800704700BF0368DA6822F49072DA60036854
:1024A8005A6922F001025A61202380F83A307047B5
:1024B8002DE9F84304460368196921F44051C268BC
:1024C8000A431A61826803691A43436942EA0301AD
:1024D8000268D36823F4B05323F00C030B43D36092
:1024E8000368596921F4407182690A435A61066890
:1024F8005A4B9E4258D1FFF729F800EB800000EBB9
:10250800800063689B00B0FBF3F9554DA5FB0929D2
:102518004FEA59194FEA0919FFF718F800EB80003C
:1025280000EB800063689B00B0FBF3F8FFF70EF840
:1025380000EB800000EB800063689B00B0FBF3F3C6
:10254800A5FB03235B09642707FB13884FEA0818D8
:1025580008F13208A5FB08384FEA581808F0F008C7
:10256800C844FEF7F3FF00EB800000EB80006368CF
:102578009B00B0FBF3F9FEF7E9FF00EB800000EBEE
:10258800800063689B00B0FBF3F3A5FB03235B09A2
:1025980007FB13973F013237A5FB0735C5F34315F2
:1025A8004544B560BDE8F883FEF7C0FF00EB800046
:1025B80000EB800063689B00B0FBF3F9284DA5FB96
:1025C80009294FEA59194FEA0919FEF7AFFF00EB3D
:1025D800800000EB800063689B00B0FBF3F8FEF717
:1025E800A5FF00EB800000EB800063689B00B0FB58
:1025F800F3F0A5FB00304009642707FB10884FEA79
:10260800081808F13208A5FB08284FEA581808F0FE
:10261800F008C844FEF78AFF00EB800000EB80005A
:1026280063689B00B0FBF3F9FEF780FF00EB8000C6
:1026380000EB800063689B00B0FBF3F0A5FB003063
:10264800400907FB10973F013237A5FB0725C5F363
:1026580043154544B560BDE8F88300BF0038014024
:102668001F85EB51704700BF10B5044658B390F86A
:10267800393013F0FF0F04D1002380F83830FFF70A
:10268800F1FF242384F839302368DA6822F40052F1
:10269800DA602046FFF70CFF23681A6922F490429B
:1026A8001A6123685A6922F02A025A612368DA6893
:1026B80042F40052DA600020E063202384F83930C5
:1026C80084F83A3010BD012010BD00BF70B582B04B
:1026D80004460D46134690F83A00C0B220283BD174
:1026E80000293BD0002A3BD094F83820012A39D061
:1026F800012284F83820A162A3850026E6632222FD
:1027080084F83A20626B19499162626B1849D16268
:10271800626B18491163626B56632168606B043100
:102728002A4600F0E7F8019623681A6801925A6869
:102738000192019A84F83860DA6842F48072DA60AB
:1027480023685A6942F001025A6123685A6942F0C3
:1027580040025A61304606E0022004E0012002E00F
:10276800012000E0022002B070BD00BF85270008EC
:10277800C9270008D9270008704700BF08B5436A71
:102788000268126812F0200F13D10022DA851A6845
:10279800D16821F48071D1601A68516921F0010172
:1027A80051611A68516921F040015161202283F872
:1027B8003A201846FFF7E0FF08BD00BF704700BF8A
:1027C80008B5406AFFF7FAFF08BD00BF704700BFB1
:1027D80010B5446A23685B6903F0800294F83930C5
:1027E800DBB2212B05D122B10023E3842046FFF779
:1027F80047FE23685B6903F0400294F83A30DBB285
:10280800222B05D122B10023E3852046FFF742FEA3
:10281800E36B43F01003E3632046FFF7D7FF10BDD7
:1028280070B4C46B056C012606FA05F5656004688A
:1028380063604368102B04D103689A600368D96009
:1028480003E0036899600368DA6070BC704700BFF2
:1028580010B4034600283CD0026820498A420AD8AE
:102868001F4911441F4AA2FB010109098900196483
:102878001D4ADA6309E01D4911441A4AA2FB010105
:102888000909890019641A4ADA63022283F82120A7
:1028980019680A6822F47F5222F030025C6898684E
:1028A8000443D86804431869044358690443986981
:1028B8000443D869204302430A6000209862D86222
:1028C800186358639863012283F8212083F8200055
:1028D80000E001205DF8044B704700BF0704024088
:1028E800F8FFFDBFCDCCCCCC00000240F8FBFDBF0B
:1028F8000004024038B5044690F82000012831D081
:10290800012084F8200094F82100012825D1022014
:1029180084F821000020A0632068056825F00105DF
:1029280005602046FFF77CFFE36A2BB123681A682D
:1029380042F00E021A6009E023681A6822F00402C5
:102948001A6023681A6842F00A021A6023681A6833
:1029580042F001021A60002038BD002384F82030BC
:10296800022038BD022038BD38B5C36B1B6801682A
:102978000C68026C042595401D4200F09D8014F0FF
:10298800040F00F099800B6813F0200F03D10B6837
:1029980023F004030B600368A84A934243D9783AAA
:1029A80093423CD01432934237D01432934231D000
:1029B800143293422BD01432934225D014329342CE
:1029C8001FD01432934219D002F56272934213D089
:1029D800143293420ED01432934208D014329342E8
:1029E80002D14FF480421BE04FF4802218E04FF4EC
:1029F800806215E0402213E0042211E04FF080626B
:102A08000EE04FF480020BE04FF4802208E04FF410
:102A1800804205E04FF4806202E0402200E0042298
:102A2800874B5A6042E0874A93423CD01432934223
:102A380037D01432934231D0143293422BD014320F
:102A4800934225D0143293421FD01432934219D0A6
:102A580002F56272934213D0143293420ED01432AC
:102A6800934208D01432934202D14FF480421BE0C3
:102A78004FF4802218E04FF4806215E0402213E002
:102A8800042211E04FF080620EE04FF480020BE068
:102A98004FF4802208E04FF4804205E04FF4806252
:102AA80002E0402200E00422674B5A60C36A002B10
:102AB80000F0C380984738BD022595401D4200F0BC
:102AC800A18014F0020F00F09D800B6813F0200F16
:102AD80006D10B6823F00A030B60012380F821302C
:102AE8000368564A934243D9783A93423CD0143209
:102AF800934237D01432934231D0143293422BD0C0
:102B08001432934225D0143293421FD01432934288
:102B180019D002F56272934213D0143293420ED048
:102B28001432934208D01432934202D14FF4005227
:102B38001BE04FF4003218E04FF4007215E0202239
:102B480013E0022211E04FF000720EE04FF4001281
:102B58000BE04FF4003208E04FF4005205E04FF468
:102B6800007202E0202200E00222354B5A6042E067
:102B7800344A93423CD01432934237D014329342B1
:102B880031D0143293422BD01432934225D01432D0
:102B980093421FD01432934219D002F562729342C5
:102BA80013D0143293420ED01432934208D0143208
:102BB800934202D14FF400521BE04FF4003218E068
:102BC8004FF4007215E0202213E0022211E04FF0CA
:102BD80000720EE04FF400120BE04FF4003208E0F0
:102BE8004FF4005205E04FF4007202E0202200E0AA
:102BF8000222154B5A60002380F82030836AE3B123
:102C0800984738BD082505FA02F21A4215D014F083
:102C1800080F12D00B6823F00E030B60C26B016C17
:102C2800012303FA01F15160836380F82130002306
:102C380080F82030036B03B1984738BD800002400C
:102C48000004024008000240000002400F4B1A68CE
:102C580042F001021A6059680D4A0A405A601A681F
:102C680022F0847222F480321A601A6822F48022D8
:102C78001A605A6822F4FE025A604FF41F029A60E2
:102C88004FF00062034B9A60704700BF001002408B
:102C98000000FFF800ED00E0F0B589B03E4EF369A2
:102CA80043F40033F361F36903F400330093009BAA
:102CB800102005210622FEF773FF1020FEF7A2FF61
:102CC800112005210722FEF76BFF1120FEF79AFF5E
:102CD800324D334B2B604FF416536B600024AC60BD
:102CE800EC602C610C236B61AC612846FFF7BCFCDF
:102CF800736943F001037361736903F0010301937E
:102D0800019BB36943F00403B361B36903F004039F
:102D18000293029BF36943F40033F361F36903F40C
:102D280000330393039B0123069304230493022394
:102D3800059303230793A6F58436304604A9FEF7C6
:102D480099FF082304930594304604A9FEF792FFDF
:102D5800144E154B33607460B4608027F76034619B
:102D680074612023B361F4613046FFF771FD6E632F
:102D780075620E4E0E4B336010237360B460F760BB
:102D880034617461B461F4613046FFF761FD2E630C
:102D9800756209B0F0BD00BF00100240FC020020BF
:102DA80000440040E40000206C000240A40200201F
:102DB8008000024030B597B01F4BDA6942F4802298
:102DC800DA61DA6902F480220092009A5A6942F0C4
:102DD80001025A615B6903F001030193019B174DDE
:102DE80006954FF4E13307930024089409940A9454
:102DF80008230B930C940D9406A8FFF735FC6B6918
:102E080043F080036B614FF48063029301230493C2
:102E18000223039303230593094802A9FEF72AFF17
:102E2800084B1C60084A9A605C6090221A60702205
:102E38001C3B5A6017B030BD0010024000480040EB
:102E4800000C01401C000240044800402DE9F04FEE
:102E580089B0814B9A6942F004029A619A6902F03A
:102E680004020192019A9A6942F008029A619A69E9
:102E780002F008020292029A9A6942F010029A61DC
:102E88009B6903F010030393039B002305930693A8
:102E98004FF00208CDF81C804FF0200A0DEB0A0411
:102EA80044F810AD6D4F38462146FEF7E3FE402347
:102EB800049338462146FEF7DDFE4FF0800BCDF82F
:102EC80010B038462146FEF7D5FE4FF480630493D0
:102ED800634D28462146FEF7CDFE4FF40063049368
:102EE80028462146FEF7C6FE4FF48056049628462B
:102EF8002146FEF7BFFE049606F1804606F57846A1
:102F080030462146FEF7B6FECDF810803046214601
:102F1800FEF7B0FE4FF00109CDF814900423049396
:102F280038462146FEF7A6FE102304933046214674
:102F3800FEF7A0FECDF810A030462146FEF79AFE17
:102F480003230593CDF8109028462146FEF792FEFC
:102F5800CDF8109030462146FEF78CFE08230493E6
:102F680028462146FEF786FECDF8108028462146E1
:102F7800FEF780FE1023049328462146FEF77AFECA
:102F8800CDF810A028462146FEF774FE04230493CA
:102F980028462146FEF76EFE082304933046214654
:102FA800FEF768FE0423049330462146FEF762FECE
:102FB800CDF814804023049328462146FEF75AFE94
:102FC800CDF810B028462146FEF754FE4FF4807A1B
:102FD800CDF810A028462146FEF74CFECDF810B0DB
:102FE80030462146FEF746FECDF810903846214679
:102FF800FEF740FECDF8108038462146FEF73AFE2F
:10300800CDF810A030462146FEF734FE4FF4007389
:10301800049330462146FEF72DFE4FF48063049357
:1030280030462146FEF726FE4FF4005304933846F7
:103038002146FEF71FFE4FF480430493384621468D
:10304800FEF718FE4FF40043049338462146FEF776
:1030580011FE09B0BDE8F08F00100240000C0140DD
:10306800001001402DE9F04F99B0754B9A6942F470
:1030780000629A619A6902F400620192019A9A695F
:1030880042F400529A619B6903F400530293029B35
:103098006C4EDFF8B891C6F80090002474604FF0C9
:1030A8002008C6F808804FF4FA6BC6F80CB03461F3
:1030B8007461B4613046FEF7CBFB10231693179466
:1030C800304616A9FEF700FD60230F931094119463
:1030D80008271297139414944FF4007315933046ED
:1030E8000FA92246FEF708FC30460FA90422FEF776
:1030F80003FC30460FA93A46FEF7FEFB4FF4006387
:1031080008934FF4806309930A94CDF82C800C94AB
:103118000D940E9430460DEB0801FEF7ABFC4A4DBA
:10312800DFF82CA1C5F800A06C60C5F80880C5F8C8
:103138000CB02C616C61AC612846FEF789FBCDF8B8
:10314800588080231793284616A9FEF7BDFC0494DF
:1031580018A9052341F8543D2846FEF70DFB6023C6
:103168000F93109411941297139414944FF40073BE
:10317800159328460FA92246FEF7BEFB28460FA93D
:103188000422FEF7B9FB28460FA93A46FEF7B4FB1E
:103198004FF4006308934FF4806309930A94CDF8C1
:1031A8002C800C940D940E9428460DEB0801FEF724
:1031B80061FCDAF8443023F40043CAF84430D9F803
:1031C800443023F40043C9F8443028462146FEF72A
:1031D8000FFC28460421FEF70BFC28463946FEF76B
:1031E80007FC28462146FEF733FC28460421FEF753
:1031F8002FFC28463946FEF72BFC30462146FEF7C1
:10320800F7FB30460421FEF7F3FB30463946FEF75C
:10321800EFFB30462146FEF71BFC30460421FEF743
:1032280017FC30463946FEF713FC2B6801221A6357
:1032380033681A6842F001021A6019B0BDE8F08FCD
:1032480000100240AC0100203C030020002C01408B
:10325800003401402DE9F04387B0414EB36943F48F
:103268000073B361B36903F400730093009B3D4C92
:103278003D4B23604FF48073A3600025E5606561D2
:103288004FF44023E36165604FF00508C4F81080EF
:103298002046FFF761F8354B5A6842F480225A609D
:1032A80006A94FF4C02341F8043D2046FEF736FC3A
:1032B800012304930E2202920393204602A9FEF7EB
:1032C800CBFE029502270397204602A9FEF7C4FE0B
:1032D80004970B27029703230393204602A9FEF7BE
:1032E800BBFE4FF00C09CDF8089004230393204649
:1032F80002A9FEF7B1FECDF80890CDF80C80204663
:1033080002A9FEF7A9FE23689A6842F480729A60BF
:103318009A6842F001029A60736943F0010373618D
:10332800736903F001030193019B114B1D60C3F8FE
:103338000480104A9A60104ADA6040F6A2221A60A5
:103348001A6842F001021A60384629462A46FEF7F2
:1033580027FC3846FEF756FC07B0BDE8F08300BFEF
:1033680000100240740200200024014000000140C7
:10337800080002404C240140E8020020F0B585B066
:10338800274B9A6942F480629A619B6903F48063CF
:103398000093009B234C244B23604FF48073A3605D
:1033A8000023E36063614FF46022E26163600526F5
:1033B80026612046FEF7D0FF012303930F220192D6
:1033C8000293204601A9FEF747FE0D23019302252B
:1033D8000295204601A9FEF73FFE03950A230193B3
:1033E80003270297204601A9FEF736FE019504231C
:1033F800029320460DEB0301FEF72EFE019702967D
:10340800204601A9FEF728FE23689A6842F48072D4
:103418009A609A6842F001029A6005B0F0BD00BF58
:1034280000100240280100200028014030B597B064
:1034380002250C9501231093102311931395002452
:1034480014944FF4601315930CA8FDF757FD0F2340
:103458000793089509944FF480630A930B9407A87F
:103468002946FDF78DFF01954FF44043039301A8CA
:10347800FEF716FDFEF754F8084BA3FB0020800961
:10348800FEF7CCFB0420FEF7DFFB4FF0FF302146B0
:103498002246FEF785FB17B030BD00BFD34D621042
:1034A8002DE9F04F83B0FEF7A3FD9F4CA36943F0CD
:1034B8000103A361A36903F001030193019B0320A6
:1034C800FEF75CFB6FF00B0000210A46FEF768FB75
:1034D8006FF00A0000210A46FEF762FB6FF0090050
:1034E80000210A46FEF75CFB6FF0040000210A4643
:1034F800FEF756FB6FF0030000210A46FEF750FB6B
:103508006FF0010000210A46FEF74AFB4FF0FF303A
:1035180000210A46FEF744FBFFF788FF636923F0A2
:1035280001036361FFF792FCFFF79CFDFFF792FE32
:10353800FFF724FFFFF73EFC7C4820210122FEF71D
:10354800A5FC7B48FEF764FE7A48FEF761FE082476
:10355800794E642504E034702846FEF769FD013C85
:10356800002CF8DA4FF0000A734B83F800A0734878
:1035780004210122FEF78AFCFFF78EFB704871498F
:103588000422FFF7A3F801226F4B1A70D34601E01B
:10359800C346A2460520FEF74BFD6A4B1B881BB2AB
:1035A800B3F57A7F0CDC674B1B881BB213F57A7F67
:1035B80003DB644B1B881BB200E0644B984601E0B8
:1035C8004FF47A78624BC3F800805E4B5B881BB27D
:1035D800B3F57A7F0BDC5B4B5B881BB213F57A7F04
:1035E80003DB584B5E8836B203E0584E01E04FF4D7
:1035F8007A76584B1E600022574B1A60574F38682E
:10360800FCF76AFF42A3D3E90023FCF7CBFF04468B
:103618000D464046FCF760FF3FA3D3E90023FCF7C3
:10362800C1FF02460B4620462946FCF709FEFDF776
:1036380053FA804638604A4F3868FCF74DFF34A388
:10364800D3E90023FCF7AEFF04460D463046FCF7ED
:1036580043FF31A3D3E90023FCF7A4FF02460B463E
:1036680020462946FCF7ECFDFDF736FA3860FCF7F2
:1036780033FF00223B4BFCF795FF06460F464046BA
:10368800FCF72AFF0022374BFCF78CFF04460D4657
:103698003046394622462B46FCF7D0FD80468946FF
:1036A8000022314BFDF70EFA80B9404649461CA36B
:1036B800D3E90023FDF7E8F928B940464946FDF764
:1036C8000BFA804604E0DFF8848001E04FF47A7852
:1036D8003046394622462B46FCF7B2FD04460D46D5
:1036E8000022214BFDF7EEF900283FD1204629465C
:1036F8000BA3D3E90023FDF7C7F928B920462946CB
:10370800FDF7EAF9044633E0104C31E0AFF30080EE
:10371800CDCCCCCCCCCCEC3F9A9999999999B93F1E
:103728000000000000408FC0001002400008014067
:103738007402002028010020C4000020000C014071
:10374800FC0200207C030020BC00002018FCFFFFC6
:103758009803002084030020040000208803002030
:10376800900300200000E03F00408F404FF47A743F
:103778000220414600F018FC0320214600F014FC0A
:103788000AF132039C4215DAAAF1320A544511DDD6
:103798000BF1320398450DDAABF1320BD84509DD50
:1037A8003A4B1B68042B05D8C8F10002384B1A6045
:1037B800384B1C6000F0FEFB37480221FEF75EFB29
:1037C800F8B10022354B1A70334D022428462146A1
:1037D800FEF754FB0028F9D10024314B1C70314B03
:1037E8001C702F4E642504E034702846FEF720FC38
:1037F8000134072CF8DD284820210022FEF746FB7B
:10380800FEE7294B1D6828462849FDF739FB58B1C2
:1038180028462749FDF752FB30B10522204B1A7084
:103828000822204B1A70B3E628462149FDF728FBE9
:1038380058B128461F49FDF741FB30B10522184B06
:103848001A700122174B1A70A2E628461949FDF78B
:1038580017FBA0B10024134B1C70104B1C70104EAA
:10386800642504E034702846FEF7E2FB0134072C97
:10387800F8DD094820210022FEF708FBFEE70023B7
:10388800074A1370074A137082E600BF040000203D
:10389800C8000020C000002000080140BC00002033
:1038A800C4000020A80000201800002000001042DA
:1038B800000004420000F8412DE9F8430222844B3D
:1038C8005A60844B1B68B3F57A7F3BDA0133814A2F
:1038D8001360814B998889B2804A1068014401EBD2
:1038E800D17149101160D98889B27D4A10680144A4
:1038F80001EBD17149101160198889B2794A1068B1
:10390800014401EBD17149101160598889B2764A96
:103918001068014401EBD17149101160598989B2CD
:10392800724A1068014401EBD171491011601A897B
:1039380092B26F4B19680A4402EBD27252101A60A5
:10394800BDE8F8836B4B1E886B4BA3FB06135B0922
:10395800642202FB13639BB223BB684F3868FCF7F1
:10396800CDFD53A3D3E90023FCF71CFE04460D4606
:10397800594B988980B2FDF7DDF9FCF7BFFD4EA3DE
:10398800D3E90023FCF70EFE4DA3D3E90023FCF78F
:1039980009FE02460B4620462946FCF751FCFDF776
:1039A800C3F838604C4B588980B2504B1C68001BD8
:1039B800FCF792FD44A3D3E90023FCF7F3FD0022B2
:1039C8000023FDF761F880B1434B588980B2001B92
:1039D800FCF782FD3CA3D3E90023FCF7E3FD0022BA
:1039E800474BFDF751F8B8B90FE03B4B588980B207
:1039F800001BFCF771FD34A3D3E90023FCF7D2FDCB
:103A08000022404BFDF75EF830B93F4B1B68052B91
:103A180002D83E4B1B782BB93D4B5A6C22F400421E
:103A28005A6404E03A4B5A6C42F400425A642A4BF6
:103A3800188980B22E4B1C68001BFCF74DFD22A391
:103A4800D3E90023FCF7AEFD00220023FDF71CF8A4
:103A580080B1214B188980B2001BFCF73DFD1AA3E9
:103A6800D3E90023FCF79EFD0022254BFDF70CF857
:103A7800C0B90FE0184B188980B2001BFCF72CFD69
:103A880011A3D3E90023FCF78DFD00221D4BFDF7A0
:103A980019F838B91C4B1B68052B03D81B4B1B782E
:103AA800002B39D11B4B5A6C22F400425A6438E07F
:103AB8002B8716D9CEF7EF3FF5E4E827181C9B3F74
:103AC800FCA9F1D24D62503F7B14AE47E17A943F96
:103AD80000000240A4000020E80200200C000020A2
:103AE8000800002014000020100000201C00002006
:103AF80020000020CC0000201F85EB51180000207A
:103B080000002EC000002E4004000020BC00002051
:103B180000340140002C01408E4B5A6C42F40042A4
:103B28005A648D4B9A6812F0200F14BF00220122AC
:103B3800996811F0400F14BF002101219B6813F010
:103B4800800F14BF00200120844B9C6814F4806F00
:103B580014BF002501259C6814F4006F14BF0027CA
:103B680001279B6813F4805F01EB400302EB4303DA
:103B78007B4CE25C7B4B1A601A6802F102021A6005
:103B88001868794981FB0082A2EBE07202EB4202DD
:103B98004FEA4202C2EB00021A600CBF0222002266
:103BA8003A4405EB4202A05C704A1060106802308B
:103BB8001060106881FB0091A1EBE07101EB4101FD
:103BC8004900411A11601B68694A908880B26949A6
:103BD8000968441AD18889B2674802688A1A052B8D
:103BE80018D8DFE803F003070A0D1013A21A634B75
:103BF8001A6012E0614B1C600FE0604B1C600CE027
:103C08005E4B1A6009E05D4B1A6006E0121B5B4BC5
:103C18001A6002E00022594B1A600136B6B2584BBE
:103C28001E80584B1B78ABB15749A1FB0621090BE5
:103C3800564A1278013291FBF2F002FB10124AB98F
:103C480096FBF3F203FB12664EB951481021FEF7BA
:103C580023F904E04E4810210022FEF717F94D4BD6
:103C68001A68404B1B68052B1AD8DFE803F00307D6
:103C78000B0E111515465242002614E05642154601
:103C8800002210E0564200250DE0554200260AE0C9
:103C980055421646002206E016465242002502E02A
:103CA8000022154616463C4B1868304B1B68052BFE
:103CB8001ED8DFE803F003080D1115190746404226
:103CC8004FF0000C17E0C0F1000C0746002012E08E
:103CD800C0F1000C00270EE047424FF0000C0AE04C
:103CE80047428446002006E084464042002702E01E
:103CF800002007468446274B1968002950DD274BCA
:103D08001968184B1C680534174B83FB0493A3EB05
:103D1800E47303EB43035B00E31A052B6FD8DFE87A
:103D280003F003070B0E11150B46494200246BE004
:103D38004C420B46002167E04C42002364E04B42B2
:103D4800002461E04B420C4600215DE00C464942EC
:103D5800002359E0002C0140000C014000100140F4
:103D6800A0490008B0000020ABAAAA2AB800002089
:103D7800E80200200C00002008000020D0000020ED
:103D8800CC000020C40000205917B7D1A80000209B
:103D980000080140C0000020C8000020AC0000203E
:103DA800784B19684B42784C246804F10108774C29
:103DB80084FB0894A4EBE87404EB44046400C4EBAB
:103DC8000804052C04D8DFE804F01E070A0E1317B0
:103DD80000210B460C4617E00C46002114E00C4667
:103DE8001946002310E01C460B46214600240BE030
:103DF8001C460B46002107E01C46002304E0002176
:103E08000B460C4600E0002426441D4401EB020842
:103E18005F4B1B68002B2ADD5E4B1A685E4B1C68E3
:103E280005345A4B83FB0493A3EBE47303EB43037E
:103E38005B00E31A052B47D8DFE803F003070B0EF6
:103E4800111513465242002143E051421346002205
:103E58003FE0514200233CE05342002139E0534205
:103E68001146002235E011465242002331E0494B09
:103E78001A68534248490C680134444981FB04914B
:103E8800A1EBE47101EB41014900611A052904D84D
:103E9800DFE801F01E070A0E131700221346114629
:103EA80017E01146002214E011461A46002310E0DC
:103EB800194613460A4600210BE01946134600220C
:103EC80007E01946002304E000221346114600E0EB
:103ED800002161443B44024406F57A7640F2C670FC
:103EE800864203DC0A2EB8BF0A2601E040F2C676F5
:103EF8002A48466305F57A7540F2C670854203DCA8
:103F08000A2DB8BF0A2501E040F2C675234885632B
:103F180008F57A7440F2C670844203DC0A2CB8BFF4
:103F28000A2401E040F2C6741C48C46301F57A71A2
:103F380040F2C670814203DC0A29B8BF0A2101E0B9
:103F480040F2C6711648416303F57A7340F2C671B0
:103F58008B4203DC0A2BB8BF0A2301E040F2C67388
:103F68000F498B6302F57A7240F2C6739A4203DCFA
:103F78000A2AB8BF0A2201E040F2C672084BDA6387
:103F8800BDE8F883AC000020B0000020ABAAAA2A44
:103F9800C8000020B4000020B80000200034014010
:103FA800002C0140AFF30080014B23F8101070473C
:103FB8000004002030B583B0144C20460021642250
:103FC80000F0A2F812490A884B888888C98800B28C
:103FD800009009B2019120460E4912B21BB200F0BE
:103FE8009BF80D4B5B6873B90B4C236823F00103F6
:103FF8002360064D284600F0B3F86060E56023684A
:1040080043F00103236003B030BD00BF9C030020D0
:1040180000040020A84900081C000240704700BFA7
:10402800FEE700BFFEE700BFFEE700BFFEE700BFF8
:10403800704700BF704700BF704700BF08B5FDF765
:10404800E9FFFDF713FE08BD08B50248FEF78CFC32
:1040580008BD00BFE400002008B50248FEF784FC54
:1040680008BD00BFA4020020002100F004B80D4BD9
:104078005B58435004310C480C4B42189A42FFF4E9
:10408800F6AF0B4A00F003B8002342F8043B094B93
:104098009A42FFF4F9AFFEF7D9FD00F00FF8FFF7E9
:1040A800FFF97047F8490008000000208800002048
:1040B8008800002014040020FFF7FEBF70B50E4BE7
:1040C8000E4D0024ED1AAD101E46AC4204D056F831
:1040D800242090470134F8E700F03CFC084D094BD8
:1040E8000024ED1AAD101E46AC4204D056F8242028
:1040F80090470134F8E770BDF0490008F04900081E
:10410800F4490008F049000802440346934202D0EB
:1041180003F8011BFAE770470EB400B54FF40271BB
:104128009CB0ADF814106FF00041049107914FF660
:10413800FF711DABADF81610084953F8042B029017
:104148000690086802A9019300F06EF8029B00220D
:104158001A701CB05DF804EB03B0704784000020AF
:10416800034613F8012B002AFBD1181A01387047AF
:104178002DE9F0478D688146AB420C4692461F46B2
:1041880043D38B8913F4906F3DD0266809690222C6
:10419800C1EB0608666906EB460696FBF2F608F1DF
:1041A80001023A44964238BF16465B050FD53146A0
:1041B80000F022FB054698B12169424600F0B4FAA6
:1041C800A38923F4906343F08003A38113E032466C
:1041D80000F066FB054670B94846216900F0C8FA48
:1041E8000C23C9F80030A3894FF0FF3043F0400397
:1041F800A381BDE8F087256166614544C8EB0606E2
:104208002560A6603D46AF4200D23D462A4620685A
:10421800514600F092FAA36800205B1BA360236854
:104228001D442560BDE8F0872DE9F0439DB0039358
:104238008B8907461C060D4616460CD50B6953B9E3
:10424800402100F0D9FA2860286110B90C233B609E
:10425800C7E040236B610023099320238DF82930A0
:1042680030238DF82A3033461C4613F8012B1AB92F
:10427800B4EB06090FD002E0252AF5D1F8E7384655
:10428800294632464B46FFF773FF013000F0A48001
:10429800099B4B4409932378002B00F09D80002351
:1042A8004FF0FF3204930793059206938DF853302D
:1042B8001A9304F101094D4E4C46304621780522E7
:1042C80000F024FA09F10109049B28B1861B01209A
:1042D800B04003430493EEE7D90644BF20228DF88B
:1042E80053201A0744BF2B228DF8532022782A2AFC
:1042F80002D0079B21460EE0039A111D1268039114
:10430800002A01DB079204E0524243F002030792BD
:10431800049301340AE00C4622780131303A092A24
:1043280003D80A2000FB0323F5E7079323782E2BF5
:1043380019D163782A2B09D1039B02341A1D1B68F3
:104348000392002BB8BF4FF0FF330BE0611C002332
:104358000C4622780131303A092A03D80A2000FB9A
:104368000323F5E70593224E21783046032200F017
:10437800CDF930B1861B4020B040049B0134034383
:10438800049321781B480622661C8DF8281000F03B
:10439800BDF988B1184B33B9039B073323F00703E2
:1043A8000833039314E003AB0093384604A92A4664
:1043B800124BAFF3008007E003AB0093384604A923
:1043C8002A460E4B00F08EF8B0F1FF3F804603D02E
:1043D800099B4344099346E7AB895B0601D40998D6
:1043E80001E04FF0FF301DB0BDE8F083BA49000886
:1043F800C0490008C44900080000000079410008CD
:104408002DE9F84315461F468A680B6906469A4205
:10441800A8BF13462B6091F843200C46DDF8208096
:104428000AB101332B602368990602D52B68023341
:104438002B60236813F006091DD094F843302268D6
:10444800003318BF012392061FD5E118302081F8E8
:1044580043005A1C94F845102244023382F8431052
:1044680013E03046394604F119020123C0470130F0
:1044780007D009F10109E2682B68D31A9945F0DBE6
:10448800DBE74FF0FF30BDE8F8833046394604F1EA
:104498004302C0470130F4D023682A6803F00603BA
:1044A800E168042B08BFC2EB01052369A2680CBFB1
:1044B80025EAE57500259A42C4BFC3EB0203ED184F
:1044C8004FF00009A9450ADA3046394604F11A02C4
:1044D8000123C0470130D4D009F10109F2E70020D7
:1044E800BDE8F8832DE9FF470E7E80466E2E0C4608
:1044F80091469A460C9D01F1430000F0A58011D821
:10450800632E22D009D8002E00F0AF80582E40F03C
:10451800BF8081F845607B4A4FE0642E1ED0692E2B
:104528001CD0B5E0732E00F0A48009D86F2E2BD0D4
:10453800702E40F0AD800B6843F020030B6038E02C
:10454800752E21D0782E34D0A2E02B6801F14207D5
:104558001A1D1B682A6081F842309DE022682B688A
:1045680012F0800F03D01A1D2A601D6805E051065D
:10457800F9D51A1D2A60B3F90050002D39DA2D2318
:104588006D4284F8433034E022682B6812F0800FC3
:1045980003D01A1D2A601D6804E05206F9D51A1DB9
:1045A8002A601D88237E574A6F2B14BF0A230823CD
:1045B8001BE07823544A84F845302368296813F0AF
:1045C800800F01F104062E6001D00D6802E05F063D
:1045D800FBD50D88DE0744BF43F0200323601DB9D7
:1045E800236823F0200323601023002184F843105C
:1045F80001E0444A0A236668002EA66003DB2168AE
:1046080021F00401216005B96EB104F14201B5FB46
:10461800F3F603FB1655555D0F4601F8015935466B
:10462800002EF4D100E00746082B0AD12368DD07E5
:1046380007D5626823699A4203DC302307F8013CF6
:10464800013FC01B20612CE009682B6811F0800F26
:10465800626904D0191D29601B681A6005E04906C3
:10466800F8D5191D29601B681A80002323610746A5
:1046780017E02B681A1D2A601F683846FFF770FD7F
:1046880063682061984288BF23612369636005E0FD
:1046980004F1420784F8426001232361002384F86F
:1046A8004330CDF800A04046214603AA4B46FFF709
:1046B800A7FE013002D14FF0FF301FE040464946C7
:1046C8003A462369D0470130F5D023689B0705D4C3
:1046D800E068039B9842B8BF18460FE00025E268DF
:1046E800039BD31A9D42F3DA4046494604F1190266
:1046F8000123D0470130DED00135F0E704B0BDE832
:10470800F08700BFCB490008DC49000810B5C9B2E2
:1047180002449042034605D01C7801308C42F8D1FF
:10472800184610BD002010BD10B50023934203D0D9
:10473800CC5CC4540133F9E710BD814270B501D394
:1047480000230EE08C18A042FAD28518134613F104
:10475800FF3305D351426618F65C2944CE54F6E778
:1047680070BD934203D0CC5CC4540133F9E770BDEB
:1047780030B500293CD051F8042C0B1F1D49002AE4
:10478800B8BF9B180A680C4612B95A600B6030BD56
:1047980093420DD219685818904203D15A581144BF
:1047A800426819605A60236030BD994203D80A46AE
:1047B80051680029F9D1146815199D420AD11B685E
:1047C8002344D0188842136012D108680344136048
:1047D8004B680CE002D90C23036030BD18681C1824
:1047E8008C4203D10C6849682044186059605360B2
:1047F80030BD00BFD800002070B5CD1C25F00305E2
:1048080008350C2D38BF0C25002D06463FDB8D42A0
:104818003DD3214B1C6818462146A1B10B685B1B90
:104828000ED40B2B03D90B60CC18CD501FE08C4253
:1048380002D1626802601AE04B6863600C4616E0B9
:104848000C464968E9E7154C23681BB9304600F067
:104858004DF820602946304600F048F8431C0146D0
:1048680015D0C41C24F0030484420AD1256004F145
:104878000B00231D20F00700C31A0BD05A42E25048
:1048880070BD3046611A00F031F80130EED10C23CA
:104898003360002070BD00BFD8000020D400002085
:1048A800F8B5064614460D4621B91146BDE8F8404C
:1048B800FFF7A2BF1AB9FFF75BFF2046F8BD00F06B
:1048C80025F8A0420ED230462146FFF795FF07464D
:1048D80050B129462246FFF727FF30462946FFF701
:1048E80047FF01E02846F8BD3846F8BD38B5064C04
:1048F800002305460846236000F012F8431C02D145
:10490800236803B12B6038BD1004002051F8040C53
:10491800002802DA04390B5818440438704700009C
:10492800094A136863B118446946884202D810607E
:1049380018467047054B0C221A604FF0FF3070473D
:10494800034B1360EFE700BFDC00002010040020D9
:1049580018040020F8B500BFF8BC08BC9E46704794
:0C496800F8B500BFF8BC08BC9E467047C4
:1049740002030405060708090A0B0C0D0E0F10109C
:104984000102000000000000000000000102030416
:1049940006070809000000000102030400000201E8
:1049A4000405030025693B25693B25693B25690A04
:1049B4000D0000004300232D302B2000686C4C00B8
:1049C400656667454647003031323334353637380B
:1049D4003941424344454600303132333435363769
:0C49E40038396162636465660000000001
:0449F0000D020008AC
:0449F400E9010008CD
:1049F80000A24A0464000000D0070000D0070000AD
:104A0800D0070000D007000000002042D0070000B7
:104A1800D0070000000000000000000000000000B7
:104A2800000000000000000000000000000000007E
:104A380000000000B8490008000000000000000065
:104A4800000000000000000000000000000000005E
:104A5800000000000000000000000000000000004E
:104A6800000000000000000000000000000000003E
:084A78000000000024000020F2
:04000005080040713E
:00000001FF
